:020000040000FA
:02000000402896
:1000800008308316810083128501831604308500B1
:100090008312860183160030860083128C018D0145
:1000A0008E018F01742289229E22B3220C157422A4
:1000B000C8220C1174220D178922C8220D1389221F
:1000C0008D158922C8228D1189220E179E22C822E1
:1000D0000E139E22C8225722131E6B289030140242
:1000E000031D5E295722131E6B2814089200572205
:1000F000131E6B28B93012070318D92837301202A3
:10010000031D85288C1774226B2838301202031DBA
:100110008C280C1774226B2839301202031D932887
:100120008C1674226B283A301202031D9A280C1682
:1001300074226B283B301202031DA1288C157422F7
:100140006B283C301202031DA8280C1574226B2862
:100150003D301202031DAF288C1474226B283E30F0
:100160001202031DB6280C1474226B283F301202B1
:10017000031DBD288D1789226B2840301202031DF4
:10018000C4280D1789226B2841301202031DCB2889
:100190008D1689226B2842301202031DD2280D16BB
:1001A00089226B2843301202031DD9288D1589221C
:1001B0006B2844301202031DE0280D1589226B289C
:1001C00045301202031DE7288D1489226B28463022
:1001D0001202031DEE280D1489226B2847301202EB
:1001E000031DF5288E179E226B2848301202031D2E
:1001F000FC280E179E226B2849301202031D03298A
:100200008E169E226B284A301202031D0A290E16F2
:100210009E226B284B301202031D11298E159E223F
:100220006B284C301202031D18290E159E226B28D4
:100230004D301202031D1F298E149E226B284E3052
:100240001202031D26290E149E226B284F30120223
:10025000031D2D298F17B3226B2850301202031D66
:1002600034290F17B3226B2851301202031D3B298A
:100270008F16B3226B2852301202031D42290F162B
:10028000B3226B2853301202031D49298F15B32264
:100290006B2854301202031D50290F15B3226B280E
:1002A00055301202031D57298F14B3226B28563084
:1002B0001202031D6B280F14B3226B288030140226
:1002C000031D6B285722131E6B2814089200572217
:1002D000131E6B28B93012070318C92937301202D0
:1002E000031D75298C1374226B2838301202031DEC
:1002F0007C290C1374226B2839301202031D8329C8
:100300008C1274226B283A301202031D8A290C12B7
:1003100074226B283B301202031D91298C11742228
:100320006B283C301202031D98290C1174226B2893
:100330003D301202031D9F298C1074226B283E3021
:100340001202031DA6290C1074226B283F301202E2
:10035000031DAD298D1389226B2840301202031D25
:10036000B4290D1389226B2841301202031DBB29C9
:100370008D1289226B2842301202031DC2290D12F0
:1003800089226B2843301202031DC9298D1189224D
:100390006B2844301202031DD0290D1189226B28CD
:1003A00045301202031DD7298D1089226B28463053
:1003B0001202031DDE290D1089226B28473012021C
:1003C000031DE5298E139E226B2848301202031D5F
:1003D000EC290E139E226B2849301202031DF329CB
:1003E0008E129E226B284A301202031DFA290E1229
:1003F0009E226B284B301202031D012A8E119E2271
:100400006B284C301202031D082A0E119E226B2805
:100410004D301202031D0F2A8E109E226B284E3083
:100420001202031D162A0E109E226B284F30120254
:10043000031D1D2A8F13B3226B2850301202031D97
:10044000242A0F13B3226B2851301202031D2B2ACA
:100450008F12B3226B2852301202031D322A0F1260
:10046000B3226B2853301202031D392A8F11B32295
:100470006B2854301202031D402A0F11B3226B283F
:1004800055301202031D472A8F10B3226B285630B5
:100490001202031D6B280F10B3226B28A0309100AD
:1004A000A0309000900B522A910B502A0800051999
:1004B000572A073097000000970B5B2A08309500F9
:1004C00094010E3097000000970B632A0310940CE0
:1004D00005199417950B612A131612309700970B84
:1004E0006F2A051D131208000C1806148C188614A8
:1004F0000C1906158C1986150C1A06168C1A8616F8
:100500000C1B06178C1B86170512000005168601AA
:1005100008000D1806148D1886140D1906158D196E
:1005200086150D1A06168D1A86160D1B06178D1BBD
:100530008617851000008514860108000E18061421
:100540008E1886140E1906158E1986150E1A0616A3
:100550008E1A86160E1B06178E1B861705100000B6
:100560000514860108000F1806148F1886140F1939
:1005700006158F1986150F1A06168F1A86160F1B69
:1005800006178F1B86178511000085158601080048
:1005900010309800C0301930C0309A009A0BCE2A23
:0A05A000990BCC2A980BCA2A080018
:02400E00F13F80
:00000001FF
